:100000000C946B000C9488000C9488000C9488006D
:100010000C9488000C9488000C9488000C94880040
:100020000C9488000C9488000C9488000C94880030
:100030000C9488000C9488000C9488000C94880020
:100040000C9488000C9488000C94DA000C948800BE
:100050000C94BA130C947C130C9488000C948800B4
:100060000C94B3020C9418130C9416140C9488007E
:100070000C9488000C9488000C9488000800000000
:10008000BE922449123EABAAAA2ABECDCCCC4C3E8D
:1000900000000080BEABAAAAAA3E00000000BF007C
:1000A0000000803F0000000000084178D3BB438778
:1000B000D1133D190E3CC3BD4282AD2B3E68EC828C
:1000C00076BED98FE1A93E4C80EFFFBE01C4FF7F11
:1000D0003F000000000011241FBECFEFD8E0DEBFBC
:1000E000CDBF12E0A0E0B1E0E6EDF6E302C005907E
:1000F0000D92A03FB107D9F714E0A0EFB2E001C024
:100100001D92AC31B107E1F70E949B060C94691B6C
:100110000C940000382FFB0190E08F709070232F1B
:100120002F700A9714F4205D01C0295C2183832F6E
:1001300082958F708A3010F4805D01C0895C808365
:100140000895F8948091F00281FF02C080E006C01B
:100150008091F00282608093F00281E0789488239D
:1001600081F38091F2028823E1F3F8943091B00397
:1001700020E008C0FD01EF54FC4F8081A055BC4F2A
:100180008C932F5FA22FB0E08091F20290E0019754
:10019000A817B9077CF38091F20281508093F20294
:1001A0007894F8948091F0028D7F8093F002789497
:1001B000832F08951F920F920FB60F9211245F9311
:1001C0006F937F938F939F93AF93BF93809113030C
:1001D00090911403019690931403809313038091DC
:1001E000130390911403892B31F484E290E09093EF
:1001F000140380931303809113039091140365E01B
:1002000070E00E94C01A892B09F045C08091150347
:1002100081608093150380911303909114036AE029
:1002200070E00E94C01A892BB1F58091150382609D
:1002300080931503809113039091140362E370E09F
:100240000E94C01A892B39F5809115038460809330
:100250001503809113039091140364E670E00E94EB
:10026000C01A892BC1F4809115038860809315030F
:1002700080915B0390915C03A0915D03B0915E035C
:100280000196A11DB11D80935B0390935C03A09325
:100290005D03B0935E03BF91AF919F918F917F916A
:1002A0006F915F910F900FBE0F901F9018959C015A
:1002B00081E080938F03F999FECF32BD21BDF89A7A
:1002C00040B510928F03FB9A81E080938F03F999D8
:1002D000FECF2F5F3F4F32BD21BDF89A20B510925F
:1002E0008F03FB9A942F80E030E0282B392BC90133
:1002F0000895282F80918E038530E0F7F894E091DF
:100300008E0383E0E89FF0011124E158FC4F9083B5
:10031000E0918E03E89FF0011124E058FC4F208308
:10032000E0918E03E89FF0011124EF57FC4F6083AA
:1003300080918E038F5F80938E0378948091F40276
:1003400084608093F402FB9A0895FF920F931F93A9
:100350008C01F62E672F0E947901C80101966F2D3E
:100360000E9479011F910F91FF90089580E090E025
:100370006091F8020E94790181E090E06091F902B9
:100380000E9479016091FA027091FB0282E090E094
:100390000E94A5016091FC027091FD0284E090E052
:1003A0000E94A5016091FE027091FF0286E090E03C
:1003B0000E94A501609100037091010388E090E024
:1003C0000E94A50160910203709103038AE090E00E
:1003D0000E94A50160910403709105038CE090E0F8
:1003E0000E94A50160910603709107038EE090E0E2
:1003F0000E94A501609108037091090380E190E0DB
:100400000E94A50160910A0370910B0382E190E0C4
:100410000E94A50160910C0370910D0384E190E0AE
:100420000E94A50160910E0370910F0386E190E098
:100430000E94A5018EEF93E0609112030E94790162
:10044000609110037091110388E190E00E94A50172
:1004500008952F923F924F925F926F927F928F9268
:100460009F92AF92BF92CF92DF92EF92FF920F9343
:100470001F933B017A01A0E0B0E0BC01CD010E94D6
:10048000551920E030E040E857E30E94281A20E0A8
:1004900030E040EA50E40E94281A5B016C0100E061
:1004A00010E0C801B7010E9455191B012C01C601BB
:1004B000B50120E030E44CE156E40E94281A7B01AB
:1004C0008C01C601B50120E030E040E050EC0E9414
:1004D000281A20E030E040EA50E40E9458189B01BE
:1004E000AC01C801B7010E94BC187B018C01C2019C
:1004F000B10120E030E543EC57E40E94BC189B01B9
:10050000AC01C801B7010E94BC180E94E8197B0128
:100510008C0188249924C401B3010E945519A801B3
:1005200097010E94BC1823E333E948E853E40E9492
:10053000571820E030E048EC52E40E94281A0E944C
:100540002419CB011F910F91FF90EF90DF90CF9076
:10055000BF90AF909F908F907F906F905F904F90E3
:100560003F902F9008951F920F920FB60F92112473
:10057000EF92FF920F931F932F933F934F935F93AD
:100580006F937F938F939F93AF93BF93EF93FF935B
:1005900040917C004F702091260330912703809179
:1005A000780090917900820F931F90932703809396
:1005B0002603809128038F5F80932803809128036E
:1005C000803449F5473020F080917C00807F0AC05C
:1005D00080917C00807F80937C0090917C00842FB0
:1005E0008F5F892B80937C00A42FB0E0809126033D
:1005F00090912703FD01EE0FFF1FEA5EFC4F9183F0
:100600008083A75DBC4F80E48C93109228031092E6
:1006100027031092260380917A00806480937A00E9
:10062000433009F498C0443038F4413009F446C0EE
:10063000423008F078C00DC0453009F4C6C04530DE
:1006400008F49FC0463009F4E4C0473009F03DC1CA
:1006500005C1609116037091170380E090E00E943D
:1006600055197B018C01609100037091010380E0BA
:1006700090E00E9455199B01AC01C801B7010E948E
:1006800057187B018C01609106037091070380E08D
:1006900090E00E9455199B01AC01C801B7010E946E
:1006A000BC1820E030E04AE754E40E94281A0E9477
:1006B0002419709336036093350307C160911803C2
:1006C0007091190380E090E00E9455197B018C0124
:1006D000609104037091050380E090E00E94551939
:1006E0009B01AC01C801B7010E9457187B018C0126
:1006F000609106037091070380E090E00E94551915
:100700009B01AC01C801B7010E94BC1820E030E099
:100710004AE754E40E94281A0E942419709338036F
:1007200060933703D2C080911A0390911B038150CC
:10073000904758F080911A0390911B038050904984
:1007400020F480913D038D7F03C080913D03826042
:1007500080933D03BAC080911C0390911D0381508A
:10076000904758F080911C0390911D038050904950
:1007700020F480913D038E7FEBCF80913D0381601B
:10078000E7CF80911E0390911F038150914738F469
:1007900080911E0390911F038050914118F482E0D4
:1007A00090E80EC080911E0390911F0360910C038E
:1007B00070910D0340910E0350910F030E94290286
:1007C00090933C0380933B0380C0809120039091E1
:1007D00021038150914738F48091200390912103A7
:1007E0008050914118F482E090E80EC0809120037F
:1007F00090912103609108037091090340910A03CD
:1008000050910B030E94290290933A03809339037D
:100810005CC0609122037091230380E090E00E940D
:1008200055197B018C016091FA027091FB0280E006
:1008300090E00E9455199B01AC01C801B7010E94CC
:10084000BC1820E030E84BE356E40E94281A0E94CE
:100850002919709332036093310337C060912403E8
:100860007091250380E090E00E9455197B018C0176
:100870006091FC027091FD0280E090E00E945519A9
:100880009B01AC01C801B7010E9457187B018C0184
:100890006091FE027091FF0280E090E00E94551985
:1008A0009B01AC01C801B7010E94BC1820E030E0F8
:1008B0004AE754E40E94281A0E9424197095619511
:1008C0007F4F7093340360933303FF91EF91BF9197
:1008D000AF919F918F917F916F915F914F913F91D8
:1008E0002F911F910F91FF90EF900F900FBE0F90DF
:1008F0001F90189585B1807F85B984B1807F84B9B8
:100900005F9A80E02DEF922F9A95F1F78F5F8A30F2
:10091000D1F72C9A26E0822F8A95F1F785B12C9891
:10092000922F9A95F1F72C9A922F9A95F1F795B10B
:10093000807F9F70892B2C98922F9A95F1F75F9862
:100940002A95F1F795B1907F95B994B19F6094B9CC
:1009500008955E980E947A0487FDFCCF0E947A0475
:1009600008951F93182F0E94A9045E9A5F9885B17D
:10097000807F85B995B1812F82958F70892B85B93C
:100980002C9A96E0892F8A95F1F72C98892F8A95D1
:10099000F1F785B1807F85B985B11F70812B85B94D
:1009A0002C9A892F8A95F1F72C989A95F1F71F9137
:1009B00008951F93182F0E94A9045E985F9885B12F
:1009C000807F85B995B1812F82958F70892B85B9EC
:1009D0002C9A96E0892F8A95F1F72C98892F8A9581
:1009E000F1F785B1807F85B985B11F70812B85B9FD
:1009F0002C9A892F8A95F1F72C989A95F1F71F91E7
:100A00000895282FDB01F8948091F00280FF02C046
:100A100080E006C08091F00281608093F00281E066
:100A20007894882381F31EC0F8940CC08091F10261
:100A3000E82FF0E09D91E057FC4F90838F5F80930B
:100A4000F10221508091F102803210F4222371F7DB
:100A50008091C10080628093C10078948091F102FE
:100A60008032E1F3222301F7F8948091F0028E7F27
:100A70008093F00278940895DF92EF92FF920F93A3
:100A80001F93DF93CF9300D0CDB7DEB7F82EE92EBA
:100A9000A82FB92FFD0101900020E9F73197DE2E34
:100AA000D81A282F392FC901FC012AE090E003C091
:100AB000819128279F5F9D15D8F3822F8E010F5FAC
:100AC0001F4FB8010E948A0081E060E071E00E943F
:100AD000010582E062E071E00E9401058D2D6F2D1D
:100AE0007E2D0E94010581E065E071E00E94010514
:100AF00082E0B8010E94010582E067E071E00E9497
:100B000001050F900F90CF91DF911F910F91FF90F2
:100B1000EF90DF900895282F81E080938F03F9995B
:100B2000FECF8EEF93E092BD81BDF89A80B5109212
:100B30008F03FB9A80931203863619F4222309F45B
:100B400052C08AE091E00E943C0586E68093120341
:100B500084E68093F90289E18093F80289E191E6C5
:100B60009093FB028093FA028BEA90E89093FD0247
:100B70008093FC0280EE97E09093FF028093FE0248
:100B800083EF96E1909301038093000326E636E617
:100B900030930303209302038AEA9AE190930503BA
:100BA0008093040330930703209306032FE23DE074
:100BB000309309032093080382E69FE290930B038E
:100BC00080930A0330930D0320930C0390930F033B
:100BD00080930E0380E39AE29093110380931003B5
:100BE0000E94B601089587E291E00E943C0584E6E8
:100BF0008093F90289E18093F80282E090E00E94FC
:100C000057019093FB028093FA0284E090E00E94E7
:100C100057019093FD028093FC0286E090E00E94D1
:100C200057019093FF028093FE0288E090E00E94BB
:100C3000570190930103809300038AE090E00E94A3
:100C4000570190930303809302038CE090E00E948D
:100C5000570190930503809304038EE090E00E9477
:100C60005701909307038093060380E190E00E9470
:100C70005701909309038093080382E190E00E945A
:100C8000570190930B0380930A0384E190E00E9444
:100C9000570190930D0380930C0386E190E00E942E
:100CA000570190930F0380930E0388E190E00E9418
:100CB0005701909311038093100308950F931F938E
:100CC000CF93DF93EC010881802F90E00E94241BDA
:100CD000892B59F11981812F90E00E94241B892BC7
:100CE00021F11A3318F4912F90530BC0173418F4D4
:100CF000912F975306C0173610F090E002C0912F45
:100D000097550A3318F4802F80530BC0073418F41A
:100D1000802F875306C0073610F080E002C0802F76
:100D200087558295807F892B01C080E0DF91CF912C
:100D30001F910F9108952F923F924F925F926F9261
:100D40007F928F929F92AF92BF92CF92DF92EF925B
:100D5000FF920F931F93DF93CF93CDB7DEB7C95A9E
:100D6000D0400FB6F894DEBF0FBECDBF15B883E0FC
:100D700088B91BB88FE184B98CE387B98AEF8AB947
:100D8000429A82E0809346038FEF9FEFAFEFBFEF71
:100D90008093530390935403A0935503B093560349
:100DA0001092C00088EB8093C10080E490E09093A3
:100DB000C5008093C4001092F5029FEE9093B80096
:100DC0008091B9008C7F8093B90085E08093BC004E
:100DD000909311045F9885B1807F85B984B18F604D
:100DE00084B95E9880E593EC0197F1F728EA31E643
:100DF000C9010197F1F785B1836085B92C9A86E026
:100E0000982F9A95F1F72C98982F9A95F1F7F90168
:100E10003197F1F72C9A982F9A95F1F72C98982FF3
:100E20009A95F1F7E8E8F3E13197F1F72C9A982FCA
:100E30009A95F1F72C98982F9A95F1F7F901319737
:100E4000F1F728982C9A982F9A95F1F72C988A9573
:100E5000F1F788E20E94D9048CE00E94D90486E070
:100E60000E94D90481E00E94D90480E80E94D9043C
:100E700080E00E94B10410928F0310928E0380E4F0
:100E800080937C008EE880937A0010927B008FEF35
:100E900080937E001092270310922603109228035D
:100EA00080917A00806480937A00789410923E0357
:100EB0008FEF9FEFAFEFBFEF8093600390936103DD
:100EC000A0936203B09363031092570310925803E8
:100ED0001092590310925A0389E08093640383E4CB
:100EE00091E00E943C0580E00E948B051092140363
:100EF000109213031092150383E084BD81E0809368
:100F00006E0083EC87BD8DE085BD82EA8093800012
:100F100088E18093810084E690E09093870080933D
:100F200086008091F90290E0909389008093880078
:100F30008091F80290E090938B0080938A008091DA
:100F400081008160809381004424772466245524A5
:100F50000FE1802E912C8C0E9D1E20E330E02C0F93
:100F60003D1F2F5E3F4FCC55DF4F39832883C45A36
:100F7000D04001C0442460914603687F60934603DB
:100F800039E1371570F561606093460380913F0346
:100F90009091400390934C0380934B0380914103C5
:100FA000909142039093480380934703855C94405B
:100FB00030F488E993E0909348038093470380914D
:100FC0004703909148038058974030F088E498E0B8
:100FD000909348038093470310924A031092490369
:100FE00043C080915B0390915C03A0915D03B0913D
:100FF0005E03209153033091540340915503509167
:101000005603821B930BA40BB50B0397A105B105E7
:10101000E4F462606093460380914D0390914E0327
:1010200090934C0380934B0380914F039091500316
:10103000909348038093470380915103909152030A
:1010400090934A03809349030FC064606093460302
:1010500010924C0310924B0310924A0310924903D2
:1010600010924803109247038091F00282FD20C045
:10107000F8948091F00282FF02C080E006C0809167
:10108000F00284608093F00281E07894882381F3F9
:1010900088E0809312048DEC8093100484E08093A8
:1010A000F5028091BC00806A8093BC004424439484
:1010B0008091150380FF70C2809115038E7F80930D
:1010C0001503209176033091770340917803509176
:1010D00079032F3F8FEF38078FEF48078FEF5807BF
:1010E00069F080915B0390915C03A0915D03B091E6
:1010F0005E03281739074A075B070CF445982091CF
:101100007A0330917B0340917C0350917D032F3F04
:101110009FEF39079FEF49079FEF590769F08091CB
:101120005B0390915C03A0915D03B0915E0328176F
:1011300039074A075B070CF4449880913E0386FD0B
:10114000B8C0806480933E0390E08F7190708430CB
:10115000910509F46FC08530910584F481309105C3
:1011600031F1823091051CF4892BB9F0A2C0823094
:10117000910539F1039709F09CC02DC08630910587
:1011800009F47AC08630910584F18730910509F41D
:101190007DC0089709F08DC083C0A5E6B3E0E2E604
:1011A000F1E080E101900D928150E1F782C0A5E667
:1011B000B3E0E3E7F1E080E101900D928150E1F7C7
:1011C00078C0A5E6B3E0E4E8F1E080E101900D929B
:1011D0008150E1F76EC0A5E6B3E0E5E9F1E080E11A
:1011E00001900D928150E1F764C0A5E6B3E0E6EA14
:1011F000F1E080E101900D928150E1F7809146038A
:1012000088608093460380915B0390915C03A0917A
:101210005D03B0915E030196A11DB11D8093600333
:1012200090936103A0936203B093630386E080937D
:101230005F033FC0A5E6B3E0E7EBF1E080E101909A
:101240000D928150E1F780914603886080934603B8
:1012500080915B0390915C03A0915D03B0915E036C
:101260000696A11DB11D8093600390936103A09326
:101270006203B09363031DC0A5E6B3E0E8ECF1E0C0
:1012800080E101900D928150E1F713C0A5E6B3E033
:10129000E9EDF1E080E101900D928150E1F709C0A4
:1012A000A5E6B3E0EAEEF1E080E101900D92815015
:1012B000E1F780913E0390E08F719070833091054B
:1012C000B1F18430910534F4009781F0019709F071
:1012D000CDC01CC08730910509F458C088309105F5
:1012E00009F481C0069709F0C1C030C080915B034A
:1012F00090915C03A0915D03B0915E0318161906EE
:101300001A061B060CF0B2C081E00EC080915B0390
:1013100090915C03A0915D03B0915E030297A105DB
:10132000B1050CF4A3C082E080933E039FC080917E
:10133000570390915803A0915903B0915A038F5FBE
:101340009F4FAF4FBF4F09F070C090C0209157031F
:10135000309158034091590350915A032F3FFFEFAA
:101360003F07FFEF4F07FFEF5F0709F47FC0809152
:101370005B0390915C03A0915D03B0915E0328171D
:1013800039074A075B070CF071C04FC02091570323
:10139000309158034091590350915A032F3F6FEFFA
:1013A00036076FEF46076FEF560769F12A3F7FEF69
:1013B00037077FEF47077FEF570709F457C0809142
:1013C0005B0390915C03A0915D03B0915E032B5F82
:1013D0003F4F4F4F5F4F281739074A075B070CF005
:1013E00045C088E0A1CF2091570330915803409128
:1013F000590350915A032F3F8FEF38078FEF48075B
:101400008FEF580711F483E08FCF80915B039091A9
:101410005C03A0915D03B0915E03821B930BA40B50
:10142000B50B0297A105B10514F487E07DCF213EED
:101430009FEF39079FEF49079FEF5907B9F0809158
:101440005B0390915C03A0915D03B0915E03225E0B
:101450003F4F4F4F5F4F281739074A075B0734F458
:1014600084E080933E0385E080935F0390913E0388
:1014700097FD09C080913D03882329F410927E03D3
:10148000906890933E0390913E0397FF2FC0809108
:101490007E038530F8F080913D0380FF1BC0892FCB
:1014A0008F71823029F485E080933E0386E010C07E
:1014B000833051F0853071F0843061F0863021F056
:1014C000873011F0883031F484E080933E0382E06D
:1014D00080935F0380913D0380FF06C080917E036F
:1014E0008F5F80937E0302C010927E032091600381
:1014F0003091610340916203509163032F3FAFEF3E
:101500003A07AFEF4A07AFEF5A0709F445C0809199
:101510005B0390915C03A0915D03B0915E0328177B
:1015200039074A075B07C4F580914603877F80939C
:1015300046032E3FBFEF3B07BFEF4B07BFEF5B07F5
:1015400059F180915B0390915C03A0915D03B09190
:101550005E032F5F3F4F4F4F5F4F281739074A07F2
:101560005B07D4F480915F0380933E0310925F0386
:101570008FEF9FEFAFEFBFEF809357039093580328
:10158000A0935903B0935A0380936003909361032F
:10159000A0936203B09363038091150381FF55C04C
:1015A0008091F602863001F51092BC008091BC005B
:1015B00080688093BC00F8948091F0028B7F8093C8
:1015C000F0027894909111041092F5029093B80073
:1015D0008091B9008C7F8093B90085E08093BC0036
:1015E000909311041092F60280913103909132038E
:1015F00020911003309111038217930720F4E3E642
:10160000E61508F0639480913103909132038217BC
:10161000930710F061106A94809131039091320326
:1016200080549F4120F422E6251508F053948091C0
:1016300031039091320380549F4110F051105A941D
:10164000809115038D7F809315036CE3651510F46D
:10165000439A01C043988091150382FF50C4809142
:1016600015038B7F809315038DB79EB70C970FB62C
:10167000F8949EBF0FBE8DBFEDB7FEB7319620E543
:1016800030E02C0F3D1FADB7BEB712963C932E93A2
:10169000119700E510E0138302836BEF71E075830F
:1016A000648380913F039091400397838683809168
:1016B00041039091420391878087809143039091E9
:1016C0004403938782870E94A8158DB79EB70C9616
:1016D0000FB6F8949EBF0FBE8DBFCE01805B9F4FAB
:1016E0000E943C0590913D03ADB7BEB71A970FB667
:1016F000F894BEBF0FBEADBFEDB7FEB7319620E583
:1017000030E02C0F3D1F12963C932E9311971383BC
:1017100002836EE072E07583648380914503868363
:101720001782908711860E94A8158DB79EB70A96DA
:101730000FB6F8949EBF0FBE8DBFCE01805B9F4F4A
:101740000E943C0560915B0370915C0380915D0396
:1017500090915E03CA55DF4F688379838A839B83A8
:10176000C65AD04020913103309132034091330367
:10177000509134036091350370913603E090370344
:10178000F0903803C0903903D0903A03A0903B0307
:10179000B0903C038DB79EB746970FB6F8949EBFA6
:1017A0000FBE8DBFEDB7FEB7319680E590E08C0F90
:1017B0009D1FADB7BEB712969C938E93119713835E
:1017C0000283ACE1B2E0B583A483CA55DF4F8881C0
:1017D0009981AA81BB81C65AD04086839783A0870E
:1017E000B187338722875587448777876687F18A51
:1017F000E08AD38AC28AB58AA48A0E94A815ADB7A6
:10180000BEB756960FB6F894BEBF0FBEADBFCE01A1
:10181000805B9F4F0E943C0580E80E94D904609144
:101820005B0370915C0380915D0390915E03209156
:101830006403E22EFF2400E010E0A80197010E945B
:10184000E71A97FD85C060915B0370915C038091FE
:101850005D0390915E03A80197010E94E71A63302F
:101860007105810591050CF073C0E0903103F09093
:101870003203A0903103B0903203809133039091F2
:10188000340397FD03C000E210E002C00DE210E057
:10189000809133039091340397FF07C08091330305
:1018A000909134036CE97FEF06C0809133039091EF
:1018B000340364E670E00E94D41AC62E472F80914C
:1018C00033039091340397FF08C0809133039091C4
:1018D0003403909581959F4F04C08091330390917C
:1018E000340364E670E00E94D41A382F292FEDB734
:1018F000FEB770970FB6F894FEBF0FBEEDBF3196DE
:10190000ADB7BEB712969C928E92119781E190E08E
:101910009383828388E392E095838483C70168EE92
:1019200073E00E94C01A77836683C50168EE73E096
:101930000E94C01A9187808713870287C4864587D3
:10194000368727870E94A815EDB7FEB77096CBC0E3
:1019500060915B0370915C0380915D0390915E03E5
:10196000A80197010E94E71A63307105810591056E
:101970000CF421C160915B0370915C0380915D0365
:1019800090915E03A80197010E94E71A66307105E5
:10199000810591050CF00FC18091390390913A03B4
:1019A00082509048D1F400D000D000D0EDB7FEB7FF
:1019B0003196ADB7BEB712969C928E92119781E187
:1019C00090E0938382838FE492E0958384830E94E6
:1019D000A815EDB7FEB736965FC080913903909198
:1019E0003A0397FD03C00BE210E002C00DE210E0E5
:1019F0008091390390913A0397FF07C08091390392
:101A000090913A036CE97FEF06C080913903909181
:101A10003A0364E670E00E94D41AF62E472F8091B4
:101A2000390390913A0397FF08C080913903909150
:101A30003A03909581959F4F04C08091390390910E
:101A40003A0364E670E00E94D41A382F292F6DB74C
:101A50007EB76C5070400FB6F8947EBF0FBE6DBF5E
:101A6000EDB7FEB73196ADB7BEB712969C928E9287
:101A7000119781E190E09383828389E592E09583D9
:101A8000848317830683F0864187328723870E94E9
:101A9000A815EDB7FEB73C960FB6F894FEBF0FBE83
:101AA000EDBF80913B0390913C038250904809F533
:101AB00000D000D000D0EDB7FEB73196CE018896A9
:101AC000ADB7BEB712969C938E93119788E090E0C5
:101AD0009383828387E692E0958384830E94A8158E
:101AE000EDB7FEB736960FB6F894FEBF0FBEEDBF4A
:101AF000E1C180913B0390913C0397FD03C00BE251
:101B000010E002C00DE210E080913B0390913C0395
:101B100097FF07C080913B0390913C036CE97FEFF6
:101B200006C080913B0390913C0364E670E00E9404
:101B3000D41AF62E472F80913B0390913C0397FFD8
:101B400008C080913B0390913C03909581959F4FF5
:101B500004C080913B0390913C0364E670E00E94D6
:101B6000D41A382F292F6DB77EB76C5070400FB63E
:101B7000F8947EBF0FBE6DBFEDB7FEB73196CE01B4
:101B80008896ADB7BEB712969C938E93119788E056
:101B900090E0938382838FE692E09583848317831A
:101BA0000683F0864187328723870E94A815EDB708
:101BB000FEB73C9698CF60915B0370915C03809177
:101BC0005D0390915E03A80197010E94E71A6630B9
:101BD0007105810591050CF4F7C060915B0370916C
:101BE0005C0380915D0390915E03A80197010E94C0
:101BF000E71A69307105810591050CF0E5C0209167
:101C00003D036DB77EB76C5070400FB6F8947EBF41
:101C10000FBE6DBFEDB7FEB73196ADB7BEB712962A
:101C20009C928E92119781E190E0938382836BE77F
:101C300072E07583648380913E0390E08F719070B1
:101C40009783868380914503808711862287138638
:101C50000E94A81580914B0390914C03ADB7BEB77D
:101C60001C960FB6F894BEBF0FBEADBF0097B9F17A
:101C7000AC01405F554057FD03C02BE230E002C08D
:101C80002DE230E0EDB7FEB73A970FB6F894FEBFFD
:101C90000FBEEDBF3196CE018696ADB7BEB7129698
:101CA0009C938E93119789E090E09383828388E8D8
:101CB00092E09583848337832683CA0157FF03C04C
:101CC000909581959F4F66E070E00E94D41A7187CD
:101CD00060870E94A815EDB7FEB73A961BC000D0EA
:101CE00000D000D0EDB7FEB73196CE018696ADB7E5
:101CF000BEB712969C938E93119789E090E09383E0
:101D0000828380E992E0958384830E94A815EDB7D1
:101D1000FEB736960FB6F894FEBF0FBEEDBF8091AA
:101D20004703909148030097D1F1AC01405F5540C3
:101D300057FD03C02BE230E002C02DE230E06DB76A
:101D40007EB76A5070400FB6F8947EBF0FBE6DBF6D
:101D5000EDB7FEB73196CE018B96ADB7BEB71296F2
:101D60009C938E93119785E090E09383828386E91C
:101D700092E09583848337832683CA0157FF03C08B
:101D8000909581959F4F66E070E00E94D41A71870C
:101D900060870E94A815EDB7FEB73A96A4CE00D092
:101DA00000D000D0EDB7FEB73196CE018B96ADB71F
:101DB000BEB712969C938E93119785E090E0938323
:101DC00082838DE992E088CE60915B0370915C0321
:101DD00080915D0390915E03A80197010E94E71A2C
:101DE000693071058105910524F160915B03709163
:101DF0005C0380915D0390915E03A80197010E94AE
:101E0000E71A6B307105810591059CF400D000D074
:101E100000D0EDB7FEB73196ADB7BEB712969C9223
:101E20008E92119781E190E09383828322EA32E0DF
:101E300034C060915B0370915C0380915D0390916D
:101E40005E03A80197010E94E71A6B3071058105B6
:101E5000910584F160915B0370915C0380915D0357
:101E600090915E03A80197010E94E71A6D307105F9
:101E700081059105FCF400D000D000D0EDB7FEB78D
:101E80003196ADB7BEB712969C928E92119781E1B2
:101E900090E09383828323EB32E0358324830E9496
:101EA000A8156DB77EB76A5F7F4F0FB6F8947EBFF7
:101EB0000FBE6DBFF40101900020E9F73197E819DA
:101EC00084017401EE0EF11C05C0D8018D918D01C5
:101ED0000E94B1040E151F05C1F780EC0E94D904C1
:101EE00080EC0E94D90405E613E005C0F801819159
:101EF0008F010E94B104F3E005371F07B9F7809105
:101F0000150383FF09C080911503877F8093150314
:101F1000429802C00E94A1008091F202882309F435
:101F200024C28091B0038432A9F71FC2DE01539608
:101F3000E3EEF2E08BE001900D928150E1F71E8E0E
:101F4000913208F053C0992309F4D6C1973010F4A8
:101F500081E04CC0092F015010E00E94A100E0E395
:101F6000F0E0EC0FFD1FE10FF11D80831F5F0117F3
:101F7000A0F788A9843211F082E038C089A98B3497
:101F800009F0BAC18AA9833409F0B6C110E0E0E3D0
:101F9000F0E0EC0FFD1FE00FF11F329780818A32D5
:101FA00011F083E023C00150104080E390E08C0FDB
:101FB0009D1F800F911F0E945E06382F91E020E048
:101FC000A8014150504009C060E370E06C0F7D1FD4
:101FD000E60FF71F808128279F5FE92FF0E0E417C5
:101FE000F50794F3231709F41EC384E0805D8C8FFA
:101FF0001D8ECE0143967EC18CA9823509F078C131
:102000008DA9813409F074C1F894AFA9A053B0E050
:10201000FD01EE0FFF1FEA5EFC4F00811181A75DFD
:10202000BC4F8C917894C8AEBE01675C7F4F0E9414
:102030008A00CBAE812FBE01645C7F4F0E948A0074
:10204000802FBE01625C7F4F0E948A0021961FAEE6
:10205000219742C1833509F06CC08CA98B3409F0FB
:102060008BC08DA9863489F5C7010E9482159C0119
:10207000442737FD4095542F1216130614061506F3
:102080004CF010927603109277031092780310921E
:10209000790332C180915B0390915C03A0915D0351
:1020A000B0915E03820F931FA41FB51F8093760328
:1020B00090937703A0937803B09379030097A105D9
:1020C000B10509F419C1459A17C1803509F010C14D
:1020D000C7010E9482159C01442737FD4095542F6B
:1020E00012161306140615064CF010927A0310927D
:1020F0007B0310927C0310927D03FEC080915B03F2
:1021000090915C03A0915D03B0915E03820F931FD9
:10211000A41FB51F80937A0390937B03A0937C0345
:10212000B0937D030097A105B10509F4E5C0449A79
:10213000E3C0873509F08CC08CA9843409F0D8C07D
:102140008DA9883449F480915B0390915C03A09140
:102150005D03B0915E0307C0843409F0C9C08FEFFE
:102160009FEFAFEFBFEF8093570390935803A09377
:102170005903B0935A03C0C0833509F0B9C08DA983
:10218000803509F0B5C080915B0390915C03A0910C
:102190005D03B0915E038093530390935403A09327
:1021A0005503B0935603C7010E945E06182FCE0157
:1021B000C9960E945E06CF55DF4F1883C15AD040A2
:1021C000C056DF4F1882C05AD04090E0C056DF4F53
:1021D000A881B981C05AD0408A2B9B2B90934E0383
:1021E00080934D03CE01CC960E945E06182FCE013F
:1021F000CE960E945E06CD55DF4F1883C35AD0405D
:10220000CE55DF4F1882C25AD04090E0CE55DF4FF6
:10221000E881F981C25AD0408E2B9F2B90935003B6
:1022200080934F03CC55DF4F88819981C45AD040A9
:102230000E945E06182FC5010E945E06312E2224E0
:1022400090E082299329909352038093510354C0C4
:10225000833409F04DC08CA9833451F58DA9982F92
:1022600090538153833008F043C0913049F48091FA
:102270002403909125039093FD028093FC0215C0E6
:10228000923049F4809116039091170390930103C3
:10229000809300030AC0933041F480911803909119
:1022A000190390930503809304030E94B60124C090
:1022B0008635A9F48DA98E34D9F4809122039091AA
:1022C00023039093FB028093FA020E94B601CEAAE8
:1022D000DFAAFBE4F8AF19AECE01C3960BC082357E
:1022E00059F48DA9813421F481E00E948B0504C04A
:1022F00084EC92E00E943C054091F20220E030E044
:102300000AC0F901E055FC4F80812F5F3F4F8D30AF
:1023100011F4892F04C0922F241798F38FEF082F00
:102320000F5F10E003C00E94A1001F5F1017D8F3D9
:102330004091F20220E030E00AC0F901E055FC4F84
:1023400080812F5F3F4F8A3011F4892F04C0922F74
:10235000241798F38FEF082F0F5F10E003C00E943F
:10236000A1001F5F101798F4FACFECE2CE2E7FE4A5
:10237000D72E67E3E62EF12CEC0EFD1E50E3A52EC2
:10238000B12CAC0EBD1E23E130E0A20EB31E409175
:10239000F20220E030E00CC0F901E055FC4F8081F2
:1023A0002F5F3F4F8D3021F49F3F09F0BFCD03C019
:1023B000922F241788F38091F202803641F4F8942A
:1023C0001092F202789480ED92E00E943C0532E394
:1023D0003615F8F48DE08093640380914703909163
:1023E000480301978752954030F488E295E0909336
:1023F0004803809347038091470390914803895B8A
:10240000964050F088EB96E0909348038093470302
:1024100003C089E080936403442011F40C94BB074B
:102420008091F00282FF04C0442443940C94BB07C3
:1024300082E3861578F480915B0390915C03A09110
:102440005D03B0915E0380FD05C080914603887FE7
:102450008093460319868091F00282FDFCCF809123
:10246000F6028130B9F490E09E01275F3F4F0AC029
:10247000E92FF0E0DF01AC5EBB4F8C91E20FF31F60
:1024800080839F5F80911204981790F380911204CB
:10249000882399F584E5898787E58A8799E49B876E
:1024A0008CE28C8786E48D8781E48E879F878CE41D
:1024B000888B198ACE0109960E943C051092BC00B7
:1024C0008091BC0080688093BC00F8948091F002F9
:1024D0008B7F8093F0027894909111041092F50212
:1024E0009093B8008091B9008C7F8093B90085E00B
:1024F0008093BC00909311047CC08985DE011996FD
:10250000813451F513962D913C9114971596ED91C8
:10251000FC91169711968D919C91129764E170E051
:102520000E94C01A7093400360933F03C90164E1A5
:1025300070E00E94C01A7093420360934103CF0180
:1025400064E170E00E94C01A7093440360934303F7
:1025500088898093450306C086E489871A86CD0161
:102560000E943C0583E4898380914703909148034E
:102570009B838A838091490390914A039D838C8336
:1025800080914B0390914C039F838E8380914603EF
:102590008887F8948091F00282FF02C080E006C034
:1025A0008091F00284608093F00281E07894882327
:1025B00081F388E08093120420E030E0AE014F5FA9
:1025C0005F4FFA01E20FF31F8081F901EC5EFB4FD0
:1025D00080832F5F3F4F2830310599F78CEC809333
:1025E000100481E08093F5028091BC00806A8093A2
:1025F000BC0080914303909144038C51974058F064
:102600007394B2E2B71510F00C94BA07442442E276
:10261000742E0C94BB07EFE0E71510F030E1732E39
:102620007A940C94BA078BA9823509F013CDE4CCC7
:102630001F920F920FB60F9211242F933F934F9337
:102640008F939F93AF93BF93EF93FF9380918F03EB
:10265000882311F0FB9842C080918E03882339F4BF
:10266000FB988091F4028B7F8093F40237C04091F5
:102670007F0320918003942F80E030E0822B932B06
:1026800092BD81BD8091810380BDFA9AF99A91E053
:1026900023E01BC0929FF0011124DF01A158BC4F21
:1026A0008C91DF01A458BC4F8C93DF01A058BC4F24
:1026B0008C91DF01A358BC4F8C93DF01AF57BC4F07
:1026C0008C91E258FC4F80839F5F80918E03981716
:1026D00008F380918E03815080938E03FF91EF91D8
:1026E000BF91AF919F918F914F913F912F910F90FB
:1026F0000FBE0F901F9018951F920F920FB60F925A
:1027000011242F938F939F93AF93BF93EF93FF93D6
:102710008091F102882331F48091C1008F7D8093F4
:10272000C1001CC0809190038093C60020E008C0C7
:10273000FD01EF56FC4F8081A057BC4F8C932F5F5B
:10274000A22FB0E08091F10290E00197A817B9079D
:102750007CF38091F10281508093F102FF91EF911F
:10276000BF91AF919F918F912F910F900FBE0F90BE
:102770001F9018951F920F920FB60F9211242F934E
:102780008F939F93EF93FF932091C6008091F20265
:102790008036D9F478948091F1028032E1F3F89494
:1027A0008091F1028032B1F39091F102E92FF0E0D3
:1027B000E057FC4F86E480839F5F9093F102809105
:1027C000C10080628093C1000AC08091F202E82FAC
:1027D000F0E0E055FC4F20838F5F8093F202809100
:1027E000F3028823C9F078948091F1028032E1F3FA
:1027F000F8948091F1028032B1F38091F102E82FD8
:10280000F0E0E057FC4F20838F5F8093F1028091CE
:10281000C10080628093C100FF91EF919F918F91E1
:102820002F910F900FBE0F901F9018951F920F922F
:102830000FB60F9211242F933F938F939F93AF93D3
:10284000BF93EF93FF939091B900987F903309F471
:10285000B0C0913390F4983109F444C0993130F408
:102860009830F1F0903109F027C11DC0903209F481
:10287000D3C0983209F020C167C0983409F4CCC0A5
:10288000993438F4983309F4A0C0903409F014C195
:10289000A8C0903509F4CCC0983509F00DC1EDC041
:1028A0008091100407C08091F50281FF0BC08091D8
:1028B000100481608093BB008091BC008F7D809369
:1028C000BC0018C08091F50280FF0AC18091BC0055
:1028D00080698093BC008091F502887F8093F50227
:1028E00085E0E2C08091F50281FF08C08091140468
:1028F0008093BB008091BC0080682DC08091F50260
:1029000080FFEEC080911204882309F4C2C0809138
:1029100014048093BB008091BC0080688093BC004D
:1029200020E008C0FD01EB5EFB4F8081AC5EBB4F39
:102930008C932F5FA22FB0E08091120490E001975A
:10294000A817B9077CF32FC08091F50281FF06C05C
:102950008091BC00806A8093BC00C2C08091F50267
:1029600080FFBEC080911204882309F492C0809138
:1029700014048093BB008091BC0080688093BC00ED
:1029800020E008C0FD01EB5EFB4F8081AC5EBB4FD9
:102990008C932F5FA22FB0E08091120490E00197FA
:1029A000A817B9077CF38091120481508093120418
:1029B00097C08091BC0080698093BC008091F50233
:1029C000887F8093F50283E06FC08091BC008068AF
:1029D0008093BC008091F502887F8093F50284E0AB
:1029E00063C0209113048091120430E090E00197BD
:1029F0002817390749F48091BC008F7B8093BC0075
:102A00008091BC00806803C08091BC00806C809382
:102A1000BC001092130464C08091BC008069809354
:102A2000BC008091F502887F8093F50282E03CC073
:102A3000209113048091120430E090E00197281750
:102A4000390749F48091BC008F7B8093BC00809152
:102A5000BC00806803C08091BC00806C8093BC0087
:102A600080911304E82FF0E09091BB00EC5EFB4FE7
:102A700090838F5F8093130433C080911304E82FF9
:102A8000F0E09091BB00EC5EFB4F90838F5F8093F2
:102A900013048091BC0080698093BC008091F50292
:102AA000887F8093F50281E08093F6028091F002A6
:102AB0008B7F8093F00214C08091BC00806880936B
:102AC000BC008091F502887F8093F50286E08093B8
:102AD000F6028091F0028B7F8093F0029093F702D0
:102AE0008091BC0080688093BC00FF91EF91BF9102
:102AF000AF919F918F913F912F910F900FBE0F90AB
:102B00001F901895FC0188279927E894219120327D
:102B1000E9F3293010F02E30C8F32B3241F02D327A
:102B200039F4689404C00E94A015820F911D219170
:102B300020532A30C0F31EF4909581959F4F08953D
:102B40007AE0979F902D879F802D910D11240895F5
:102B5000AEE0B0E0EEEAF5E10C94401B0D891E8971
:102B60008F89988D97FF02C080E090E801979E833F
:102B70008D831A83098386E08C83CE014B96AC014A
:102B8000698D7A8DCE0101960E94D8154D815E81A6
:102B900057FD0AC02F813885421753070CF49A015C
:102BA000020F131FF80110822E96E4E00C945C1BB8
:102BB000ABE0B0E0EEEDF5E10C94321B3C012B01F3
:102BC0005A01FC0117821682838181FD03C06FEFD9
:102BD0007FEFC8C19AE0892E1E010894211C311C88
:102BE000F3012381F20123FD859123FF81912F01C0
:102BF000882309F4B4C1853239F423FD859123FF7C
:102C000081912F01853229F4B30190E00E94CD1704
:102C1000E7CF982FDD24CC249924FFE1FD15D0F0D7
:102C20009B3269F09C3228F4903259F0933291F43F
:102C30000EC09D3249F0903369F441E024C052E067
:102C4000D52A84E0D82A28C098E0D92A25C0E0E116
:102C5000DE2A22C0D7FC29C0892F80538A3070F425
:102C6000D6FE05C0989C902C1124980E15C0C89CC7
:102C7000C02C1124C80EF0E2DF2A0EC09E3229F4C7
:102C8000D6FC6DC140E4D42A07C09C3619F450E844
:102C9000D52A02C0983649F4F20123FD959123FF0D
:102CA00091912F01992309F0B8CF892F8554833052
:102CB00018F08052833038F444E050E0A40EB51E82
:102CC0005FE359830FC0933631F0933779F0933532
:102CD00009F056C020C0F5018081898342E050E0B0
:102CE000A40EB51E710101E010E012C0F501E080F4
:102CF000F180D6FC03C06FEF7FEF02C0692D70E05A
:102D000042E050E0A40EB51EC7010E94C2178C011C
:102D10005FE7D52214C0F501E080F180D6FC03C046
:102D20006FEF7FEF02C0692D70E042E050E0A40E2B
:102D3000B51EC7010E94B7178C0150E8D52AD3FEF3
:102D400007C01AC0B30180E290E00E94CD17CA9478
:102D50008C2D90E008171907A8F30EC0F701D7FCD7
:102D60008591D7FE81917F01B30190E00E94CD173C
:102D7000C110CA94015010400115110579F7ECC03B
:102D8000943611F0993671F5D7FE08C0F501E08050
:102D9000F1800281138144E050E00AC0F501808196
:102DA00091817C010027F7FC0095102F42E050E054
:102DB000A40EB51E5FE6D52217FF0AC01095009538
:102DC000F094E094E11CF11C011D111D80E8D82A4B
:102DD0002AE030E0A101C801B7010E94F917F82EDE
:102DE000F21840C0953729F41D2D1F7E2AE030E0EF
:102DF0001DC01D2D197F9F3661F0903720F4983546
:102E000009F0ADC00FC0903739F0983709F0A7C06E
:102E100004C028E030E00AC0106114FD146020E115
:102E200030E004C014FD166020E132E017FF08C056
:102E3000F501608171818281938144E050E008C096
:102E4000F50180819181BC0180E090E042E050E09A
:102E5000A40EB51EA1010E94F917F82EF2188FE7F3
:102E6000D82ED122D6FE0BC05EEFD522F91438F44D
:102E7000D4FE07C0D2FC05C08FEED82202C01F2DA1
:102E800001C0192DD4FE0DC0FE01EF0DF11D808192
:102E9000803319F499EED92208C01F5FD2FE05C015
:102EA00003C08D2D867809F01F5F0D2DD3FC14C053
:102EB000D0FE0FC01C1510F09F2C0BC09F2C9C0C3B
:102EC000911A1C2D06C0B30180E290E00E94CD173C
:102ED0001F5F1C15C0F304C01C1510F4C11A01C0FB
:102EE000CC2404FF10C0B30180E390E00E94CD1712
:102EF00002FF1EC001FD03C088E790E002C088E524
:102F000090E0B3010CC0802F867891F001FF02C0E1
:102F10008BE201C080E2D7FC8DE2B30190E00E9419
:102F2000CD1706C0B30180E390E00E94CD179A94BC
:102F3000F914C0F3FA94F101EF0DF11DB301808192
:102F400090E00E94CD17FF20A9F706C0B30180E2F0
:102F500090E00E94CD17CA94CC20C1F741CEF30176
:102F600066817781CB012B96E2E10C944E1BFC012C
:102F70000590615070400110D8F7809590958E0FA4
:102F80009F1F0895FC016150704001900110D8F717
:102F9000809590958E0F9F1F08950F931F93CF9349
:102FA000DF938C01EB018B8181FF1BC082FF0DC081
:102FB0002E813F818C819D812817390764F4E88137
:102FC000F9810193F983E88306C0E885F985802FAC
:102FD0000995892B31F48E819F8101969F838E8381
:102FE00002C00FEF1FEFC801DF91CF911F910F912A
:102FF0000895FA01AA27283051F1203181F1E8948F
:103000006F936E7F6E5F7F4F8F4F9F4FAF4FB1E0DB
:103010003ED0B4E03CD0670F781F891F9A1FA11DD6
:10302000680F791F8A1F911DA11D6A0F711D811DD7
:10303000911DA11D20D009F468943F912AE0269F9C
:1030400011243019305D3193DEF6CF010895462FFB
:103050004770405D4193B3E00FD0C9F7F6CF462FDC
:103060004F70405D4A3318F0495D31FD4052419345
:1030700002D0A9F7EACFB4E0A69597958795779502
:103080006795BA95C9F700976105710508959B0189
:10309000AC010A2E06945795479537952795BA9512
:1030A000C9F7620F731F841F951FA01D0895505804
:1030B000BB27AA270ED04DC13ED130F043D120F01E
:1030C00031F49F3F11F41EF433C10EF4E095E7FB99
:1030D00029C1E92F4FD180F3BA176207730784071C
:1030E000950718F071F49EF567C10EF4E0950B2E6C
:1030F000BA2FA02D0B01B90190010C01CA01A0014A
:103100001124FF27591B99F0593F50F4503E68F1A4
:103110001A16F040A22F232F342F4427585FF3CFE5
:10312000469537952795A795F0405395C9F77EF4B6
:103130001F16BA0B620B730B840BBAF09150A1F0FF
:10314000FF0FBB1F661F771F881FC2F70EC0BA0F85
:10315000621F731F841F48F4879577956795B7950D
:10316000F7959E3F08F0B3CF9395880F08F0992705
:10317000EE0F9795879508950CD0EBC0E3D040F003
:10318000DAD030F021F45F3F19F0CCC0511115C1F5
:10319000CFC0F0D098F39923C9F35523B1F3951B11
:1031A000550BBB27AA2762177307840738F09F5F68
:1031B0005F4F220F331F441FAA1FA9F333D00E2ED7
:1031C0003AF0E0E830D091505040E695001CCAF744
:1031D00029D0FE2F27D0660F771F881FBB1F261709
:1031E00037074807AB07B0E809F0BB0B802DBF01DC
:1031F000FF2793585F4F2AF09E3F510568F092C019
:10320000DCC05F3FECF3983EDCF3869577956795DD
:10321000B795F7959F5FC9F7880F911D969587958C
:1032200097F90895E1E0660F771F881FBB1F6217AB
:1032300073078407BA0720F0621B730B840BBA0B69
:10324000EE1F88F7E095089504D06894B111B5C0D9
:10325000089598D088F09F5790F0B92F9927B751CB
:10326000A0F0D1F0660F771F881F991F1AF0BA954A
:10327000C9F712C0B13081F09FD0B1E008959CC071
:10328000672F782F8827B85F39F0B93FCCF3869540
:1032900077956795B395D9F73EF49095809570959D
:1032A00061957F4F8F4F9F4F0895E89409C097FB1A
:1032B0003EF490958095709561957F4F8F4F9F4F0D
:1032C0009923A9F0F92F96E9BB279395F695879551
:1032D00077956795B795F111F8CFFAF4BB0F11F414
:1032E00060FF1BC06F5F7F4F8F4F9F4F16C08823BB
:1032F00011F096E911C0772321F09EE8872F762FF1
:1033000005C0662371F096E8862F70E060E02AF031
:103310009A95660F771F881FDAF7880F969587951D
:1033200097F9089597F99F6780E870E060E0089545
:103330009FEF80EC089500240A94161617061806CD
:103340000906089500240A941216130614060506A9
:103350000895092E0394000C11F4882352F0BB0F3A
:1033600040F4BF2B11F460FF04C06F5F7F4F8F4F9D
:103370009F4F089557FD9058440F551F59F05F3FD8
:1033800071F04795880F97FB991F61F09F3F79F087
:1033900087950895121613061406551FF2CF469509
:1033A000F1DF08C0161617061806991FF1CF86958B
:1033B0007105610508940895E894BB27662777276F
:1033C000CB0197F908950EF0A6C0B2CF6894AACFAA
:1033D000D9DFC8F39923D1F3C6F3DF93CF931F93BB
:1033E0000F93FF92C92FDD2788232AF02197660FBC
:1033F000771F881FDAF720E030E040E85FEB9FE3BB
:10340000883920F0803E30F021968F7751DEECE74E
:10341000F0E003C04DDEE9EAF0E08DD08B01BE01A3
:10342000EC01FB2E6F5771097595771F880B990B6F
:103430003EDF28E132E741E35FE316D0AF2D98018C
:10344000AE01FF900F911F91CF91DF9142DE81CFAE
:103450000BD07FCF70DF28F075DF18F0952309F0CF
:1034600061CF66CF1124A9CF85DFA0F3959FD1F35B
:10347000950F50E0551F629FF001729FBB27F00D22
:10348000B11D639FAA27F00DB11DAA1F649F662777
:10349000B00DA11D661F829F2227B00DA11D621FC6
:1034A000739FB00DA11D621F839FA00D611D221F80
:1034B000749F3327A00D611D231F849F600D211D64
:1034C000822F762F6A2F11249F5750408AF0E1F007
:1034D00088234AF0EE0FFF1FBB1F661F771F881F50
:1034E00091505040A9F79E3F510570F01BCF65CF1A
:1034F0005F3FECF3983EDCF3869577956795B7953B
:10350000F795E7959F5FC1F7FE2B880F911D969564
:10351000879597F908959F3F49F0915028F4869533
:1035200077956795B7959F5F80389F4F880F9695E1
:10353000879597F90895DF93CF931F930F93FF9289
:10354000EF92DF927B018C01689405C0DA2EEF01C7
:103550008BDFFE01E894A591259135914591559118
:10356000AEF3EF01B6DDFE019701A801DA9479F719
:10357000DF90EF90FF900F911F91CF91DF91089511
:10358000AA1BBB1B51E107C0AA1FBB1FA617B70789
:1035900010F0A61BB70B881F991F5A95A9F78095A5
:1035A0009095BC01CD01089597FB092E07260AD0FE
:1035B00077FD04D0E5DF06D000201AF47095619500
:1035C0007F4F0895F6F7909581959F4F089597FB4B
:1035D000092E05260ED057FD04D014D00AD0001CA9
:1035E00038F450954095309521953F4F4F4F5F4FA0
:1035F0000895F6F790958095709561957F4F8F4F60
:103600009F4F0895A1E21A2EAA1BBB1BFD010DC0FE
:10361000AA1FBB1FEE1FFF1FA217B307E407F50782
:1036200020F0A21BB30BE40BF50B661F771F881F5E
:10363000991F1A9469F760957095809590959B01F4
:10364000AC01BD01CF010895911109C080538A508A
:1036500028F0865C806281568650B8F708959927D5
:10366000882708952F923F924F925F926F927F9298
:103670008F929F92AF92BF92CF92DF92EF92FF9282
:103680000F931F93CF93DF93CDB7DEB7CA1BDB0B2E
:103690000FB6F894DEBF0FBECDBF09942A883988D3
:1036A00048885F846E847D848C849B84AA84B984DA
:1036B000C884DF80EE80FD800C811B81AA81B981E6
:1036C000CE0FD11D0FB6F894DEBF0FBECDBFED01FA
:0636D0000895F894FFCFFD
:1036D60024004B41002A000D0A004E464F2C4C6F29
:1036E6006164696E672064656661756C74207365D4
:1036F6007474696E6773004E464F2C4C6F61646933
:103706006E6720656570726F6D2073657474696E7F
:103716006773004E464F2C32303039313231372CF8
:10372600302E312C616E727040616E72702E6E6535
:1037360074004B6179616B20636F6E74726F6C20DD
:10374600626400286329616E727040616E72702E29
:103756006E65740049646C6520202020202020209E
:10376600202020200049646C652C20574420646981
:103776007361626C64005072657373206275747451
:103786006F6E206F6E2000507265737320627574C1
:10379600746F6E206F6666005761746368646F6746
:1037A6002077616974696E67005761746368696E32
:1037B600672E2E2E20202020200057617463686417
:1037C60067206C61746520686974005353522C2518
:1037D6003034782C253034782C2530347800534416
:1037E600522C253032782C25303278005356522C04
:1037F600256C692C253035752C25692C25692C25D9
:10380600692C25692C2569002532692E25303369F6
:1038160056202563253033692E2530326941002D27
:103826002D2D2E2D2D4320200025632532692E2592
:10383600303269432020002D2D2D2E2D2D430025BD
:10384600632532692E2530326943002575202530DF
:103856003278253032782000256325303369200000
:103866002D2D2D2D2000256325303369002D2D2D7E
:103876002D0042617474657279206372697469639C
:10388600616C00546872757374206C696D69746537
:10389600642020004552522C496E76616C696400A2
:1038A6004552522C534552494E2C4F564552464C82
:1038B6004F57004552522C4E4D45412C58000000A2
:00000001FF
